:100F8D00C108015A00015957015B08015C03422851
:030F9D00AB0000A6
:04239700438020223D
:04239B005380DF226A
:04239F006380202215
:0622DC0053B4F053B23FC1
:0722E200908000E559F02295
:0C2310005359BF1222E24359400222E25E
:06237A005359DF0222E2CC
:062380004359200222E295
:062386005359EF0222E2B0
:06238C004359100222E299
:10224F00E55C20E1064380025380FB5359F70222DD
:01225F00E29C
:10226000E55C20E1065380FD4380044359080222C7
:01227000E28B
:07235E005380EF535CFE22E7
:10214E005380F7E55930E3085380FD438004800641
:0A215E004380025380FB535CFD2216
:07236500438010435C0122DC
:07236C0043800E435C0222D6
:0C231C00535BFE5359FBE4F5B60222E2CD
:0D22E900435B014359041222E275B6FF2247
:0C232800535BFD5359FD53B40F0222E239
:0D22F600435B024359021222E243B4F0227E
:10220500535BFB435B085359FE1222DC43B4014385
:03221500B2C02232
:10227100435B04535BF74359011222DC43B40E2242
:0323AF0002227196
:0323B200022205FF
:0323B500AFB122A3
:0323B8008FB122C0
:07237300E5A0C4540FFF2296
:0F22A100EF540FC454F0FFE5A0540F4FF5A022E7
:08233E00E5A0540EC313FF22B9
:0E22CE00EF540725E0FFE5A054F14FF5A022E4
:0F228100E58054C0C4135407FFE5A054014FFF7C
:01229000222B
:1020FD00EF5406C43354E0FEEF5401FFE580543F26
:0A210D004EF580E5A054FE4FF5A04A
:0121170022A5
:10106800AE07EEB41200400302113990107AF82846
:1010780028730210B00210B00210B00210B00210B3
:10108800B00210B00210B00210B00210CD0210CDA4
:101098000210CD0210CD0210F10210F10210F1027F
:1010A80011150211150211157401A806088002C352
:1010B80033D8FCF455B1FFED60047C0180027C005C
:1010C800EF4CF5B122122373EE24F8FC7401A80446
:1010D800088002C333D8FCF45FFFED60047C018014
:1010E800027C00EF4CFF0222A112233EEE24F4FC06
:1010F8007401A804088002C333D8FCF45FFFED60D4
:10110800047C0180027C00EF4CFF0222CE12228177
:10111800EE24F1FE7401A806088002C333D8FCF45B
:101128005FFFED60047E0180027E00EF4EFF12201B
:02113800FD2296
:100DB700AD07EDB412004003020EAB900DC9F82841
:100DC7002873020DFF020DFF020DFF020DFF020D3A
:100DD700FF020DFF020DFF020DFF020E27020E2775
:100DE700020E27020E27020E53020E53020E530263
:100DF7000E7F020E7F020E7F1223B5EFFB7A00747F
:100E0700017E00A805088005C333CE33CED8F9F498
:100E1700FFEEF45AFEEF5B4E60037F01227F002254
:100E2700122373EFFB7A00ED24F8FF74017E00A80C
:100E370007088005C333CE33CED8F9F4FFEEF45A52
:100E4700FEEF5B4E60037F01227F002212233EEFFD
:100E5700FB7A00ED24F4FF74017E00A807088005E3
:100E6700C333CE33CED8F9F4FFEEF45AFEEF5B4E20
:100E770060037F01227F0022122281EFFB7A00EDBF
:100E870024F1FF74017E00A807088005C333CE3321
:100E9700CED8F9F4FFEEF45AFEEF5B4E60037F0104
:070EA700227F00227F0022E0
:101F3C00120B8EFF1223B8900001120BA7FF122276
:101F4C00A1900002120BA7FF1222CE900003120BDD
:051F5C00A7FF0220FDBB
:101F61001223B5EF120BD4122373900001EF120B61
:101F7100E612233E900002EF120BE612228190003E
:051F810003EF020BE676
:0123CB0022EF
:0123CC0022EE
:1021980090291074FFF0A3740FF0A37407F0A3F054
:0621A800E490290FF02273
:101CDD007B017A297910121F3C90290FE030E00525
:101CED001222E9800312231C90290FE030E1051226
:101CFD0022F6800312232890290FE030E2051222EC
:0B1D0D00718003122205D204D20522CF
:10208D00AE07AC05300609120DB7EF6401FD8007F0
:0C209D00AF06120DB7AD07AF04021068CB
:0123CD0022ED
:0123CE0022EC
:0123CF0022EB
:0123D00022EA
:0123D10022E9
:1015900012236512236C12231C1223281222051217
:1015A000224F90E61274A0F0000000E490E613F0E1
:1015B00000000090E61474E0F0000000E490E615EE
:1015C000F090E6047480F00000007402F000000067
:1015D0007406F0000000E4F000000090E618F0004F
:1015E00000007411F000000090E61A7409F0000089
:1015F0000012113AE490E672F090E671F0000000FB
:1016000090E6D204F000000090E6E204F0D200126E
:10161000231043B23E755957755B08755C0312235E
:041620009BD2042233
:10145600200846E5BB30E741E5AB20E13C00000053
:1014660090E690E0FC00000090E691E0FD000000B0
:10147600ECC313FCED13FDEC90E6D0F0000000AFDA
:1014860005EF90E6D1F0000000E4F5BB000000E5B2
:10149600BB30E7030080F80000300850E5BB30E7BA
:1014A60027E55A7023E5AC20E04200000090E6D024
:1014B6007402F0000000E490E6D1F0000000755AD6
:1014C6000175BB0600000022E5BB30E71FE55AB4F4
:1014D600011A00000090E6AFE06402600690E6B0F4
:0C14E600E0600690E6487406F0E4F55A59
:0114F20022D7
:1005B000E4F529F52AD204120A6A500302078C9046
:1005C000E6B9E024EE603D24DE24FD4003020690FF
:1005D000247C700302075514700302076C14700327
:1005E0000206CF24AA600302078A90E740E55BF089
:1005F000A3E55CF0E490E68AF090E6BEE090E68B3E
:10060000F002078CE490E68AF090E6BEE090E68B7C
:10061000F090E6A0E020E1F990E744E030E0051238
:1006200022E9800312231C90E744E030E105122206
:10063000F6800312232890E744E030E2051222718D
:10064000800312220590E744E030E3051223B280D4
:10065000031223AF90E740E0FF1223B8A3E0FF129C
:1006600022A1A3E0FF1222CEA3E0FF1220FD90E71B
:1006700045E030E005122365800312235E90E745D4
:10068000E030E10612236C02078C12214E02078C27
:1006900012231090E6047480F00000007402F00051
:1006A00000007406F0000000E4F000000090E69105
:1006B0007480F0000000F0000000F0000000F00086
:1006C0000000E490E68AF090E68B04F002078CE4E8
:1006D00090E68AF090E6BEE090E68BF090E6A0E02F
:1006E00020E1F990E741E09028ABF090E742E090FC
:1006F00028ACF090E740E030E00C1223869028AC64
:10070000E04403F0800A12238C9028ACE04402F00D
:100710007A287BAB7D027F171220E190E743E090BF
:1007200028ABF090E744E09028ACF090E740E03050
:10073000E10C12237A9028ACE04403F0800A1223E3
:10074000809028ACE04402F07A287BAB7D027F16D3
:100750001220E1802CC20812226090E6F574FFF0AE
:10076000E490E68AF090E68B04F08015D20812221D
:100770004F90E6F574FFF0E490E68AF090E68B0483
:0D078000F090E6A0E04480F08002D322C398
:01078D002249
:10130000120100020000004005160F8000000102DB
:1013100000010A060002000000400100090220004E
:1013200001010080320904000002FF0000000705EF
:1013300002020002000705860200020009022E00D8
:1013400001010080320904000004FF0000000705CD
:101350000202400000070504024000000705860263
:101360004000000705880240000014030000000050
:1013700000000000000000000000000000000C035E
:10138000410043004300450053002403550053002F
:1013900042002D00440049004F002D00310036006E
:1013A00041000000000000000000000000000000FC
:100FA000608028000101010101010107000000002B
:100FB00000000000070707070707070700000000F9
:100FC0000000003F010101010101010700000000D4
:100FD00000000000070707070707070700000000D9
:100FE0000000003F8F01070101010107010003021A
:100FF000020202000701070707070707F200F200D5
:101000000000003F0F010F0101010107010205006F
:10101000000000000706070707070707F000F000B9
:101020000000003F6024288700000000000000004E
:1010300000000000000000000000000000000000B0
:10104000000000000000000000000000472880E0D1
:06105000000007BA4E008B
:10113A0090E60174BAF090E6F574FFF0902880E02A
:10114A0090E6F3F0902881E090E6C3F0902882E0E0
:10115A0090E6C1F0902883E090E6C2F0902885E0FE
:10116A0090E6C0F0902886E090E6F4F075AF077438
:10117A0028F59A7400F59B759DE4E4F59EFF90E6C8
:10118A007BE090E67CF00FBF80F4E490E671F0F526
:10119A00B490E672E0547FF053B67F000000E4900A
:1011AA00E6C4F000000090E6C5F0902887E090E6DB
:1011BA00C6F0902888E090E6C7F0902889E090E68B
:1011CA00C8F090288AE090E6C9F090288BE090E673
:1011DA00CAF090288CE090E6CBF090288DE090E65B
:0A11EA00CCF090288EE090E6CDF0E6
:0111F40022D8
:10213300564A756C20303920323031354031353ACA
:0B21430033353A33310000000000008B
:101056000255214A024000000148010144010142B3
:011066000188
:102218009028B0E070069028AFE060030223031214
:03222800239222DC
:101FF1007E007F677D007B017A2879AD120C83908A
:1020010028AD7409F0E4A3F01223CB1223CC0221F2
:01201100AE20
:1020A9007D02121AF09028ADE0B40904A3E06003A0
:0C20B900021FF17D67121AF01223CC22E6
:1021AE007A287BAD7D677F017E1F121DBC7D677F08
:0621BE00007E1F0223BB9E
:10185D0012221890E6BEE0F531753302E53160577E
:10186D00C3944050058531328003753240E490E6D3
:10187D008AF090E68BE532F090E6A0E020E1F9E405
:10188D00F530E530C39532502574402530F582E4AE
:10189D0034E7F583E0FFAE330533EE7C007B0124A6
:1018AD00ADF9EC3428FAEF120BD4053080D4C3E532
:0A18BD00319532F53180A5022218A2
:1013B00090E6B8E030E745E4F531F530E530C39428
:1013C0000550247E007B01740A2530F9EE3429FA99
:1013D000120B8EFF74402531F582E434E7F583EF7C
:1013E000F00530053180D5E490E68AF090E6BEE065
:1013F00090E68BF090E6A0E04480F02290E6BEE01C
:1014000090E68BF090E6A0E020E1F990E6BEE06483
:10141000056003C20422E4F531F530E530C39405DC
:10142000502474402531F582E434E7F583E0FFE58C
:10143000307C007B01240AF9EC3429FAEF120BD43A
:101440000530053180D590E6BAE0B4CE08A3E0B40B
:05145000AC031221AE07
:011455002274
:0F22B000D3E5589546E557954540031222BF22C6
:0123D20022E8
:101FAB009028B2E0FE9028B1E07C002400F546ECCE
:101FBB003EF54545467007C28CC2A9C20522D28C9C
:031FCB00D2A92276
:0123D30022E7
:101C1E0090E6BEE090E68BF090E6A0E020E1F9E4DD
:101C2E00FF74422FF582E434E7F583E0FEEF7C008B
:101C3E007B01240FF9EC3429FAEE120BD40FBF05F9
:101C4E00E090E740E09028B1F090E741E09028B2B4
:041C5E00F0021FABC6
:0F22BF00121CDDE4F50BF50CF557F558D205228E
:10205100C205E4F50BF50CF557F558C28CC2A9532E
:0E2061008EF75389F14389011223D3021FAB7E
:101CA100E54145406019E54115417002154014C3F5
:101CB10094FFE54064809480501C12239B80173070
:101CC10004147540057541FF122397C204E4F50B16
:0B1CD100F50CF557F558300502D20461
:011CDC0022E5
:10092F0090E6B8E020E7030209E4E4F5319028B13E
:10093F00E0FFAE31053174402EF582E434E7F583E4
:10094F00EFF09028B2E0FFAE31053174402EF58202
:10095F00E434E7F583EFF0E4F530E530C394055068
:10096F00247E007B01740F2530F9EE3429FA120B27
:10097F008EFF74402531F582E434E7F583EFF005FF
:10098F0030053180D5AE31053174402EF582E43417
:10099F00E7F583E558F0E557FFAE31053174402E8A
:1009AF00F582E434E7F583EFF0A205E433FFAE31CF
:1009BF00053174402EF582E434E7F583EFF0C2057C
:1009CF00E490E68AF090E6BEE090E68BF090E6A029
:1009DF00E04480F02290E6BEE090E68BF090E6A037
:1009EF00E020E1F9C20590E6BEE064076003C204AF
:1009FF0022E4F531AF31053174402FF582E434E74D
:100A0F00F583E09028B1F0AF31053174402FF582B6
:100A1F00E434E7F583E09028B2F0E4F530E530C335
:100A2F009405502474402531F582E434E7F583E0D2
:100A3F00FFE5307C007B01240FF9EC3429FAEF122B
:100A4F000BD40530053180D5121FAB90E6BAE0B458
:0A0A5F00CE08A3E0B4AC031221AEF0
:010A6900226A
:0423A3007548012256
:1018C70012221890E6BEE0F531E4F533E5316057B2
:1018D700C3944050058531328003753240E490E669
:1018E7008AF090E68BE532F090E6A0E020E1F9E49B
:1018F700F530E530C39532502574402530F582E444
:1019070034E7F583E0FFAE330533EE7C007B01243B
:10191700C8F9EC3428FAEF120BD4053080D4C3E5AC
:07192700319532F53180A576
:01192E002296
:101A4C001548E548704B9028C8E0F5481223CDE4C2
:101A5C00F522902909E0FFE522C39F5031E52225AC
:101A6C00E024C9F582E43428F583E0F523E522254A
:101A7C00E024CAF582E43428F583E0F524547FFD94
:101A8C00E524339206AF2312208D052280C4122345
:011A9C00CE7B
:011A9D002226
:1020120090E6BEE090E68BF090E6A0E020E1F99039
:10202200E740E09028B3F090E741E09028B4F02236
:1017D2001544E544600302185C9028B3E0F5447BAD
:1017E200017A297944121F61E4FFFE74442EF582C6
:1017F200E43429F583E0FD74142EF582E43429F5EE
:1018020083E06DF97D01E4FCECC394085046E95D88
:10181200602974182FF582E43429F583E014F074FA
:10182200182FF582E43429F583E0702074142EF524
:1018320082E43429F583E06DF080009028B4E0FB67
:1018420074182FF582E43429F583EBF00CED25E0D2
:0A185200FD0F80B40EEE64047091E7
:01185C002269
:1021680090E6BEE090E68BF090E6A0E020E1F990E2
:08217800E740E09028B5F022D9
:101EB800E4FF74382FF582E43429F583E4F07440A4
:101EC8002FF582E43429F58374FFF0743C2FF582F2
:0B1ED800E43429F583E4F00FBF04D7C9
:011EE30022DC
:101993001542E542705B9028B5E0F5427B017A2958
:1019A3007938121F61E4FF74402FF582E43429F57E
:1019B30083C083C082E0FE74382FF582E43429F5B6
:1019C30083E0FDEE5DD082D083F0743C2FF582E49A
:1019D3003429F583C083C082E0FE74382FF582E496
:1019E3003429F583E0FDEE4DD082D083F00FBF04A0
:0119F300B63D
:0119F40022D0
:0423A7007547012253
:101624001547E547603DE4F5229028C7E0FFE52231
:10163400C39F507C744D2522F8E6602316E6701F84
:10164400E52225E024B7F582E43428F583E0FE544E
:101654007FFFEE30E7047D0080027D0112106805F3
:101664002280C69028B6E0F547E4F5229028C7E02A
:10167400FFE522C39F5039E52225E024B8F582E432
:101684003428F583E0FF744D2522F8A607E52225CA
:10169400E024B7F582E43428F583E0FE547FFFEEBE
:1016A40030E7047D0180027D00121068052280BCB1
:0116B4002213
:101E250090E6BEE090E68BF090E6A0E020E1F9E4D4
:101E3500FF74402FF582E434E7F583E0FEEF7C0084
:101E45007B0124B6F9EC3428FAEE120BD40FBF123D
:011E5500E0AC
:011E56002269
:0414F3008E308F3177
:1014F700E4F532E53164024530700C90E741F0E5E0
:1015070031153170021530E53164014530701690A0
:10151700E7407467F090E6BEE090E68BF0E53115A2
:101527003170021530E5314530605D90E6A0E0206E
:10153700E1F9C3E5319440E53094005004AD3180C2
:10154700027D40E4FFEFC39D5025AE320532EE75B4
:1015570083007B0124ADF9E5833428FA120B8EFE54
:1015670074402FF582E434E7F583EEF00F80D6E47C
:1015770090E68AF090E68BEDF0FFC3E5319FF531F9
:08158700E5309400F530809D71
:01158F002239
:1000800090E6B8E030E76390E6BFE0FE90E6BEE0C1
:10009000FDEDFF4E7002804D90E6BDE0FD90E6BCA8
:1000A000E04D70030214F390E6BDE0600302038AA2
:1000B00090E6BCE014600302038A7533FF753421B7
:1000C00075353375360075371E7B017AE779411235
:1000D0001A9E7B017AE779401221F0EF0490E74005
:1000E000F090E6BEE090E68BF02290E6BFE0FF9055
:1000F000E6BEE04F707790E6BDE0704D90E6BCE064
:1001000024EF6023249F603024FD603324F36034A7
:100110002472703590E6BAE064CE702DA3E064AC32
:1001200070271221AE802290E6BAE0B4CE1BA3E085
:10013000B4AC16121FF18011E49028C7F0800A7544
:1001400047018005E4902909F090E6BDE0648060F5
:100150000302038A90E6BCE06401600302038A9014
:10016000E6BAE09028AFF090E6BB02021D90E6BF31
:10017000E0600302038A90E6BDE0FE90E6BCE07C0E
:10018000002400FFEC3E600302038AEF120C5D01C5
:10019000C32001C32101C32201C32301F82F02257B
:1001A00041023351024153026161026F63028F7158
:1001B000029D7302BD74031281031D83033A840000
:1001C00000038A90E6BEE0B4650312185D90E6BCB9
:1001D000E030E0031223CC90E6BCE020E103020310
:1001E0008A90E6BAE064CE600302038AA3E064ACBE
:1001F000600302038A0221AE90E6BEE0640260035F
:1002000002038AE090E68BF090E6A0E020E1F9128C
:10021000221890E740E09028AFF090E741E0902866
:10022000B0F002221890E6BEE06407600302038A81
:10023000021C1E90E6BEE06402600302038A0220F4
:100240001290E6BEE06401600302038AE090E68B50
:10025000F090E6A0E020E1F990E740E09028B3F0CC
:100260002290E6BEE06401600302038A02216890E6
:10027000E6BEE06401600302038AE090E68BF09042
:10028000E6A0E020E1F990E740E09028B5F0229068
:10029000E6BEE06412600302038A021E2590E6BEF9
:1002A000E06401600302038AE090E68BF090E6A030
:1002B000E020E1F990E740E09028B6F02290E6BE19
:1002C000E06402600302038A9028C7E0C3940840F8
:1002D0000302038A90E6BEE090E68BF090E6A0E091
:1002E00020E1F990E740E0FF9028C7E0FE25E024F8
:1002F000B5F582E43428F583EFF090E741E0FFEEB6
:1003000025E024B6F582E43428F583EFF09028C781
:10031000807590E6BEE0644270700218C790E6BE39
:10032000E064017065E090E68BF090E6A0E020E1EB
:10033000F990E740E09028C8F02290E6BEE0640221
:100340007048902909E0C39420503F90E6BEE090A9
:10035000E68BF090E6A0E020E1F990E740E0FF9026
:100360002909E0FE25E024C7F582E43428F583EF6F
:10037000F090E741E0FFEE25E024C8F582E4342860
:0A038000F583EFF0902909E004F086
:01038A002250
:1021180090E6047480F00000007402F0000000747F
:0B21280006F0000000E4F000000022C0
:0123D40022E6
:101C6200E4F5297AE779407F40AB077D087FF87E6B
:101C72001D121AF8E4F52974402529F582E434E7A7
:101C8200F583E0FDE52975F002A4246CF97413359F
:0E1C9200F08982F583EDF00529E529B408D923
:011CA0002221
:1012B80090E678E05410FFC4540F4450F54913E405
:1012C80033F54B90E600E054E74410F0438E2012CB
:1012D8002392121590122356121C621223D1D200A7
:1012E8001220A91220511223A3121EB81223A712EA
:0812F800221812239B0223CFF0
:10206F001223D0121CA11222B0E58090E68020E04E
:0E207F0006E04408F08004E054F7F002145626
:0619F5008B5E8A5F896031
:1019FB00E4F5611221F08F62E56225E02402901379
:101A0B008AF0E4F561AF62EF3395E0FEC3E5619FC9
:101A1B00EE6480F87480985027AB5EAA5FA960854E
:101A2B006182758300120BA7FDE56175F002A4249A
:101A3B008CF9741335F08982F583EDF0056180C55F
:011A4B002278
:061B8D008E3E8F3FAC0507
:101B9300E4FDE54B6012E53EFF7E000DEE2556F5B4
:101BA30082E43555F583EFF0AE050DE5562EF5824B
:101BB300E43555F583E53FF0AF050DE5562FF58286
:101BC300E43555F583ECF0AB56AA55AF491220E145
:051BD300AF49021D8670
:0323BB00021B8D75
:0A1DBC008E388F398D3A8A3B8B3C3C
:101DC600E4F53DE53DC3953A50200539E539AE3891
:101DD6007002053814FFE53C253DF582E4353BF5F8
:0A1DE60083E0FD1223BB053D80D908
:011DF00022D0
:081AF0007A287BAD7F017E1F07
:0A1AF8008E388F398D3A8A3B8B3C03
:101B0200E4FDF53DE54B6012E538FF7E000DEE2564
:101B120056F582E43555F583EFF0AE050DE5562E08
:101B2200F582E43555F583E539F0AB56AA55AF4950
:0E1B32001220E1AB3CAA3BAD3AAF490220C500
:10078E0090E6BAE0753000F531A3E0FEEE4230900F
:10079E00E6BEE0753200F533A3E0FEEE423290E69F
:1007AE00B8E064C0600302089BE533453270030273
:1007BE00092E90E6A0E020E1F9C3E5339440E5323E
:1007CE0094005008853234853335800675340075B3
:1007DE00354090E6B9E064A3705890E6BCE0B401F1
:1007EE001BA3E0701790E6BBE030E71090E7407473
:1007FE0003F0A37401F0A37403F0806CE4F536F5F6
:10080E0037C3E5379535E5369534505CE5312537F8
:10081E00F582E5303536F583E0FF74402537F582F5
:10082E0074E73536F583EFF00537E53770D30536C7
:10083E0080CFE4F536F537C3E5379535E536953493
:10084E00501974402537F58274E73536F58374CD2B
:10085E00F00537E53770E0053680DCAD357AE77B9D
:10086E0040AF31AE30121AF8E490E68AF090E68B83
:10087E00E535F02531F531E5343530F530C3E53366
:10088E009535F533E5329534F5320207B790E6B873
:10089E00E06440600302092EE5334532700302091D
:1008AE002EE490E68AF090E68BF090E6A0E020E150
:1008BE00F990E68BE0753400F53590E6B9E0B4A317
:1008CE0036E4F536F537C3E5379535E536953450CC
:1008DE003374402537F58274E73536F583E0FFE54E
:1008EE00312537F582E5303536F583EFF00537E5FE
:1008FE003770D3053680CFAD357AE77B40AF31AE5A
:10090E0030121DBCE5352531F531E5343530F53085
:10091E00C3E5339535F533E5329534F5320208A645
:01092E0022A6
:0B11F500E54645457003D38001C3228E
:0223C100D32225
:0223C300D32223
:0823460090E6BAE0F543D32252
:10222B0090E740E543F0E490E68AF090E68B04F00B
:02223B00D322AC
:08234E0090E6BAE0F54AD32243
:10223D0090E740E54AF0E490E68AF090E68B04F0F2
:02224D00D3229A
:0223C500D32221
:0223C700D3221F
:0223C900D3221D
:100EAE00E4FF90E6B8E020E703020F8C0F0F7440CA
:100EBE002401F582E434E7F5837409F00F744024BD
:100ECE0002F582E434E7F583E4F00F74402403F571
:100EDE0082E434E7F583E4F00F74402404F582E4F1
:100EEE0034E7F5837401F00F74402405F582E43481
:100EFE00E7F5837404F00F74402406F582E434E7BA
:100F0E00F583E4F00F74402407F582E434E7F583AB
:100F1E00E4F00F74402408F582E434E7F58374FF9F
:100F2E00F00F74402409F582E434E7F58374FFF082
:100F3E000F7440240AF582E434E7F5837408F00F49
:100F4E007440240BF582E434E7F5837420F00F74BB
:100F5E0040240CF582E434E7F5837410F00F7440EE
:100F6E00240DF582E434E7F5837410F090E740EF3A
:0E0F7E00F0E490E68AF090E6BEE090E68BF09C
:010F8C002242
:100A6A0090E6B9E0120C5D0AB1100AB1110ADF145E
:100A7A000B50150A9F280A992E0A933C0AAB3F0A83
:100A8A00A5A20AA5A300000B8A120080020B8C12F1
:100A9A00092F020B8C1213B0020B8C12078E020B59
:100AAA008C120EAE020B8C90E6B8E030E70C7B019C
:100ABA007AE77940121F61020B7490E6BEE090E675
:100ACA008BF090E6A0E020E1F97B017AE779401209
:100ADA001F3C020B8CE4F52C7438252CF582E43487
:100AEA0029F583E0FF7440252CF582E434E7F58389
:100AFA00EFF0052CE52CB404DFE4F52C7440252C2A
:100B0A00F582E43429F583E0FF7444252CF582E468
:100B1A0034E7F583EFF0052CE52CB404DFE4F52C7B
:100B2A00743C252CF582E43429F583E0FF744825CA
:100B3A002CF582E434E7F583EFF0052CE52CB404B8
:100B4A00DF121EB88024E4F52C7414252CF582E4F7
:100B5A003429F583E0FF7440252CF582E434E7F567
:100B6A0083EFF0052CE52CB404DFE490E68AF090DC
:100B7A00E6BEE090E68BF090E6A0E04480F08002CA
:030B8A00C322D3B0
:010B8D002245
:10203200C0E0C083C08290E6B5E04401F0D2015313
:0F20420091EF90E65D7401F0D082D083D0E03250
:1021C400C0E0C083C0825391EF90E65D7404F0D008
:0621D40082D083D0E0324E
:1021DA00C0E0C083C0825391EF90E65D7402F0D0F4
:0621EA0082D083D0E03238
:101D1800C0E0C083C08290E680E030E70E85090FFE
:101D2800850A10851311851412800C85130F8514EC
:101D380010850911850A125391EF90E65D7410F031
:071D4800D082D083D0E0320D
:10218000C0E0C083C082D2035391EF90E65D740833
:08219000F0D082D083D0E032D0
:101D4F00C0E0C083C08290E680E030E70E85090FC7
:101D5F00850A10851311851412800C85130F8514B5
:101D6F0010850911850A125391EF90E65D7420F0EA
:071D7F00D082D083D0E032D6
:0123D50032D5
:0123D60032D4
:0123D70032D3
:0123D80032D2
:0123D90032D1
:0123DA0032D0
:0123DB0032CF
:0123DC0032CE
:0123DD0032CD
:0123DE0032CC
:0123DF0032CB
:0123E00032CA
:0123E10032C9
:0123E20032C8
:0123E30032C7
:0123E40032C6
:0123E50032C5
:0123E60032C4
:0123E70032C3
:0123E80032C2
:0123E90032C1
:0123EA0032C0
:0123EB0032BF
:0123EC0032BE
:0123ED0032BD
:0123EE0032BC
:0123EF0032BB
:0123F00032BA
:0123F10032B9
:0123F20032B8
:0123F30032B7
:0123F40032B6
:0123F50032B5
:0123F60032B4
:0123F70032B3
:0123F80032B2
:101FCE00902948EFF0F5CB8FCDAF05A3EFF0F5CA12
:101FDE008FCCE4F5C8758E19D2BDD2AFD2ADD2CAB0
:031FEE00F5632276
:0D2303009028B0E0FF9028AFE0FD021FCE53
:0323BE00AF6322E8
:10229100AD07AC06C3E49DFBE49CFFEBFD021FCE42
:05239200C2CAC2AD2229
:03002B0002192F88
:10192F00C0E0C0F0C083C082C0D075D000C000C07E
:10193F0001C002C003C004C005C006C0079028B391
:10194F00E060031217D29028B5E06003121993904C
:10195F0028C7E06003121624902909E06009902837
:10196F00C8E06003121A4CC2CFD007D006D005D002
:10197F0004D003D002D001D000D0D0D082D083D0F9
:04198F00F0D0E03282
:0A2334000001020203030404050582
:03000B00021B4095
:101B4000C0E0C0F0C0D075D000C000C004C005C067
:101B500006C0070508E508B4060B0558E5587002ED
:101B60000557750800AE57AF587C007D0A120C0867
:101B7000ED4C7008050CE50C7002050BD007D00683
:0D1B8000D005D004D000D0D0D0F0D0E0329D
:1016B500E4F528F527F526F525C203C200C202C2C6
:1016C500011212B8750D13750E00751513751612E6
:1016D500750913750A1C75131375143C7517137565
:1016E500186AD2E843D82090E668E04409F090E60D
:1016F5005CE0443DF0D2AFD207121E8990E680E04F
:1017050054F7F0538EF8C20330010512038BC20162
:101715003003291211F55024C203121F862000162A
:1017250090E682E030E704E020E1EF90E682E030E9
:10173500E604E020E0E4121EE41223C112206F80CB
:01174500C7DC
:10038B0090E6B9E0700302043C1470030204B92434
:10039B00FE700302053C24FB700302043614700349
:1003AB000204301460731460762405600302059C0C
:1003BB001223C340030205A890E6BBE024FE602293
:1003CB0014603324FD601114602224067048E50D7F
:1003DB0090E6B3F0E50E8037E51590E6B3F0E51641
:1003EB00802DE50F90E6B3F0E5108023E51190E644
:1003FB00B3F0E512801990E6BAE0FF121F10AA06BF
:10040B00A9077B01EA494B600DEE90E6B3F0EF9044
:10041B00E6B4F00205A80205A112223D0205A812BE
:10042B00234E0205A81223460205A812222B020511
:10043B00A81223C540030205A890E6B8E0247F600C
:10044B001514601924027063A200E43325E0FFA2A7
:10045B0002E4334F8041E490E740F0803F90E6BCEC
:10046B00E0547EFF7E00E0D394807C0040047D014D
:10047B0080027D00EC4EFEED4F2434F58274233E5A
:10048B00F583E493FF3395E0FEEF24A1FFEE34E612
:10049B008F82F583E0540190E740F0E4A3F090E6FF
:1004AB008AF090E68B7402F00205A80205A11223D4
:1004BB00C740030205A890E6B8E024FE60162402AC
:1004CB0060030205A890E6BAE0B40105C20002057C
:1004DB00A80205A190E6BAE0705590E6BCE0547E08
:1004EB00FF7E00E0D394807C0040047D0180027D80
:1004FB0000EC4EFEED4F2434F58274233EF583E47D
:10050B0093FF3395E0FEEF24A1FFEE34E68F82F5E7
:10051B0083E054FEF090E6BCE05480131313541F99
:10052B00FFE0540F2F90E683F0E04420F0806E80C4
:10053B00651223C9506790E6B8E024FE601A2402C6
:10054B00705B90E6BAE0B40104D200805090E6BA3A
:10055B00E0B402028047803E90E6BCE0547EFF7E12
:10056B0000E0D394807C0040047D0180027D00EC90
:10057B004EFEED4F2434F58274233EF583E493FF56
:10058B003395E0FEEF24A1FFEE34E68F82F58380F6
:10059B00081205B0500790E6A0E04401F090E6A0E9
:0405AB00E04480F0B8
:0105AF002229
:030033000223ABFA
:0423AB0053D8EF32E2
:03004300021200A6
:0300530002120096
:10120000022032000221DA000221C4000221800003
:10121000021D1800021D4F000223D5000223D60034
:101220000223D7000223D8000223D9000223DA00C8
:101230000223DB000223DC000223DD000223DE00A8
:101240000223DF000223D6000223E0000223E10094
:101250000223E2000223E3000223E4000223E5006C
:101260000223E6000223D6000223D6000223D60082
:101270000223E7000223E8000223E9000223EA0038
:101280000223EB000223EC000223ED000223EE0018
:101290000223EF000223F0000223F1000223F200F8
:1012A0000223F3000223F4000223F5000223F600D8
:0812B0000223F7000223F800FD
:101EE40090E682E030E004E020E60B90E682E03009
:101EF400E119E030E71590E680E04401F07F147EBC
:0C1F040000121BD890E680E054FEF02292
:101F860090E682E044C0F090E681F04387010000CD
:041F96000000002225
:101E890030070990E680E0440AF0800790E680E098
:101E99004408F07FDC7E05121BD890E65D74FFF0E4
:0F1EA90090E65FF05391EF90E680E054F7F0225F
:08235600E4F51ED2E9D2AF222A
:101D860090E678E020E6F9C2E990E678E04480F053
:101D9600EF25E090E679F090E678E030E0F990E61D
:101DA60078E04440F090E678E020E6F990E678E0C6
:061DB60030E1D6D2E92263
:101E5700A90790E678E020E6F9E51E702390E6787A
:101E6700E04480F0E925E090E679F08D19AF03A909
:101E770007751A018A1B891CE4F51D751E01D322FB
:021E8700C32274
:101DF100A90790E678E020E6F9E51E702590E678DF
:101E0100E04480F0E925E0440190E679F08D19AFD6
:101E110003A907751A018A1B891CE4F51D751E03A8
:041E2100D322C322E3
:03004B00020CAFF5
:100CAF00C0E0C083C082C085C084C086758600C086
:100CBF00D075D000C000C001C002C003C006C0077D
:100CCF0090E678E030E206751E06020D9990E67800
:100CDF00E020E10CE51E64026006751E07020D9907
:100CEF00E51E24FE605F14603624FE7003020D8A39
:100CFF0024FC7003020D9624086003020D99AB1AB1
:100D0F00AA1BA91CAF1D051D8F82758300120BA78F
:100D1F0090E679F0E51D65197070751E05806B9072
:100D2F00E679E0AB1AAA1BA91CAE1D8E8275830053
:100D3F00120BE6751E02E5196401704E90E678E01D
:100D4F004420F08045E51924FEB51D0790E678E0B4
:100D5F004420F0E51914B51D0A90E678E04440F000
:100D6F00751E0090E679E0AB1AAA1BA91CAE1D8E6A
:100D7F0082758300120BE6051D800F90E678E04424
:100D8F0040F0751E008003751E005391DFD007D011
:100D9F0006D003D002D001D000D0D0D086D084D0DE
:080DAF0085D082D083D0E03230
:021F1000A9071F
:101F1200AE17AF188F828E83A3E064037017AD01F2
:101F220019ED7001228F828E83E07C002FFDEC3E42
:091F3200FEAF0580DF7E007F0098
:011F3B002283
:1020C500121DF1E51E24FA600E146006240770F354
:0C20D500D322E4F51ED322E4F51ED32232
:1020E100121E57E51E24FA600E146006240770F3D1
:0C20F100D322E4F51ED322E4F51ED32216
:101BD8008E298F2A90E600E054187012E52A240115
:101BE800FFE43529C313F529EF13F52A801590E68C
:101BF80000E05418FFBF100BE52A25E0F52AE52977
:101C080033F529E52A152AAE29700215294E6005F3
:061C1800121F9A80EE226B
:101F9A007400F58690FDA57C05A3E582458370F95A
:011FAA002214
:030000000217469E
:0C174600787FE4F6D8FD75816402178DF1
:100B8E00BB010689828A83E0225002E722BBFE0265
:090B9E00E32289828A83E4932298
:100BA700BB010CE58229F582E5833AF583E0225003
:100BB70006E92582F8E622BBFE06E92582F8E2224D
:0D0BC700E58229F582E5833AF583E4932267
:100BD400BB010689828A83F0225002F722BBFE0100
:020BE400F322FA
:100BE600F8BB010DE58229F582E5833AF583E8F045
:100BF600225006E92582C8F622BBFE05E92582C8F1
:020C0600F222D8
:100C0800BC000BBE0029EF8DF084FFADF022E4CCD0
:100C1800F875F008EF2FFFEE33FEEC33FCEE9DEC99
:100C2800984005FCEE9DFE0FD5F0E9E4CEFD22EDDF
:100C3800F8F5F0EE8420D21CFEADF075F008EF2F29
:100C4800FFED33FD4007985006D5F0F222C398FD1A
:050C58000FD5F0EA22B7
:100C5D00D083D082F8E4937012740193700DA3A326
:100C6D0093F8740193F5828883E47374029368603A
:060C7D00EFA3A3A380DF3A
:101A9E008B308A318932E4F538F539E5371537AEB2
:101AAE0036700215364E6033AB33AA34A935120B9D
:101ABE008EFFAB30AA31A9320539E539AC38700248
:101ACE00053814F5828C83EF120BE6EF60CD7401AE
:101ADE002535F535E43534F53480C0AB30AA31A95F
:021AEE003222A2
:1021F000E4FFFE120B8E600C0FEF70010E09E97008
:05220000F20A80EF224C
:100C8300EF4E6012EF60010EEDBB010B89828A8388
:100C9300F0A3DFFCDEFA2289F05007F709DFFCA995
:0C0CA300F022BBFEFCF309DFFCA9F022EC
:101752000216B5E493A3F8E493A34003F68001F2E2
:1017620008DFF48029E493A3F85407240CC8C33398
:10177200C4540F4420C8834004F456800146F6DF67
:10178200E4800B0102040810204080900F8DE47E5B
:10179200019360BCA3FF543F30E509541FFEE4935C
:1017A200A360010ECF54C025E060A840B8E493A323
:1017B200FAE493A3F8E493A3C8C582C8CAC583CA4E
:1017C200F0A3C8C582C8CAC583CADFE9DEE780BE06
:011067000088
:00000001FF
